:1018000050C084C069C068C067C066C065C064C09D
:1018100063C062C061C060C05FC05EC05DC05CC0CC
:101820005BC05AC059C00403090412036F00620070
:101830006400650076002E0061007400100348000B
:101840004900440042006F006F0074001201100153
:1018500000000008C016DF050001010200010902B6
:101860002200010100800A090400000103000000B9
:10187000092101010001222100070581030800C898
:101880000600FF0901A101150026FF00750885016A
:1018900095060921B20201850295830922B202014F
:1018A000C00011241FBECFE5D4E0DEBFCDBF10E0E5
:1018B000A0E6B0E0E4ECFFE102C005900D92AA368C
:1018C000B107D9F710E0AAE6B0E001C01D92A73A2F
:1018D000B107E1F737D375C393CFA82FB92F80E0B5
:1018E00090E041E050EA60956F5F58F42D9138EF39
:1018F00082279795879510F0842795273F5FC8F337
:10190000F3CF0895EADF8D939D930895CF93CFB7DA
:10191000CF93829BFECF829B09C0829B07C0829B94
:1019200005C0829B03C0829B01C0A3C0DF93C0910E
:101930008A00DD27CF56DF4F829B02C0DF91EBCFBD
:101940002F930F931F9300B32FEF02FB20F94F93B8
:101950003F9310B34FEF012702FB21F93BE031C069
:101960004E7F012F10B3216028C0102F4D7F2260C1
:10197000000000B329C04B7F2460012F000010B38A
:101980002BC010B3477F28602AC04F7E00B3206170
:101990002CC04F7D10B320622FC04F7B00B320645A
:1019A00032C0422700B349934FEF0000102712FBCB
:1019B00020F910B31C70C9F1297F91F2012702FBB5
:1019C00021F900B3237F89F2315058F1102712FB1F
:1019D00022F910B3277E79F2012702FB23F92F7C2D
:1019E00081F200B3102712FB24F92F7971F200C0A5
:1019F00010B3012702FB25F92F7359F200C000B381
:101A0000102712FB26F9223040F200C010B3012744
:101A100002FB27F9243028F64F77206810B3000026
:101A2000F9CF10E41ABF002719C03B503195C31BF2
:101A3000D04010E41ABF0881033CF9F00B34E9F000
:101A4000209188001981110F1213EDCF4A81441F94
:101A5000093641F10D3211F0013E29F700938F0054
:101A60003F914F911F910F912F91DF91CAB7C6FD02
:101A700050CFCF91CFBFCF91189520918F002223C7
:101A800079F310918D001123A1F53430A2F1309338
:101A90008D002093890010918A003BE0311B309328
:101AA0008A0029C000918D0001301CF50AE54F70B5
:101AB00049F43091600034FD20C000936000C1E71C
:101AC000D0E01FC030917C0034FD17C000937C0033
:101AD000CDE7D0E016C0052710E002BB1FC00527E8
:101AE00022C0052727C005272CC0052710E002BB10
:101AF00033C04AE503C042ED01C0432FC4E1D0E04A
:101B000032E011B31C60929A02B311BB5F935CE0A8
:101B100020E820FF052702BB279517951C3FD8F624
:101B200020FF0527279502BB17951C3FC0F620FF15
:101B300005272795179502BB1C3F98F620FF052720
:101B4000279517951C3F02BB70F600C0499120FFF6
:101B5000052702BB279517951C3F38F620FF052760
:101B6000279502BB17951C3F40F520FF05272795B9
:101B7000179502BB1C3F18F520FF052727951795E1
:101B80001C3F02BBF0F4242F3A9519F6037F5F91B6
:101B900002BB000010918E00110FC651D04011F011
:101BA0001093880010E41ABF046011B3137F402F14
:101BB000437F02BB11BB42BB53CF0527D2CF0527C2
:101BC000D7CF0527DCCFF89481E180935700E895C3
:101BD00081E08BBF1BBE14C20895BF92CF92DF92EB
:101BE000EF92FF920F931F93CF93DF9320918D007D
:101BF000922F935097FD38C180918A00CDE9D0E0B3
:101C0000C81BD109809189008D3209F0B3C098308A
:101C100009F028C183EC809371008AE5809360000D
:101C200010926A003881832F8076D1F089818930C3
:101C300041F48A818093620010926F008FEF90E0F0
:101C40000DC0813019F080E090E008C083E690E09C
:101C500090938C0080938B0087E090E0982F78C061
:101C60009A8110927A008981882321F410927B0056
:101C700022E067C0853019F490938E0061C08630F1
:101C800009F04AC08B81813019F48CE498E11AC0C4
:101C9000823041F48EE598E190938C0080938B0024
:101CA00092E235C08330F1F4992341F486E298E161
:101CB00090938C0080938B0094E029C0913041F484
:101CC0008AE298E190938C0080938B0092E11FC090
:101CD0009230E1F48CE398E190938C0080938B0038
:101CE00090E115C0813241F48EE998E190938C0027
:101CF00080938B0099E00BC0823241F480E898E138
:101D000090938C0080938B0091E201C090E080E47E
:101D100080936A00292F1BC0883021F421E080E9DC
:101D200090E011C0893019F49093900009C08A3076
:101D300011F421E006C08B3019F48BE480937D0010
:101D400020E08AE790E090938C0080938B00922FA4
:101D50009F3F31F437FD9E8180E880936A0007C081
:101D60008F81882321F42E81291708F4922F9093D4
:101D7000610078C080916A0087FF74C08091620022
:101D8000813019F4809370006BC0823009F068C014
:101D9000892F90916F00992371F4FE013196E980AB
:101DA000DF011196F180FD010181ED01229610E025
:101DB000822F875008C0E0906B00F0906C0000917B
:101DC0006D0010916E00792F780F70936F00682F5F
:101DD000669523E0B22E91E0C92E85E0D82EC7018A
:101DE0008F739070892B49F4F894F701B0925700E3
:101DF000E895789407B600FCFDCFF89428813981E6
:101E00000901F701C0925700E89511247894A801C0
:101E100097012E5F3F4F4F4F5F4F79018A01C901F4
:101E20008F739070892B59F4F894C9010297FC01C3
:101E3000D0925700E895789407B600FCFDCF61502A
:101E400011F02296CCCF20936B0030936C0040931E
:101E50006D0050936E0077FF05C08FEF8093620096
:101E60001092610010928D008091600084FF46C046
:101E7000609161006F3F09F441C090917100693039
:101E800008F047C01092610088E89827909371008D
:101E9000662309F447C020918B0030918C0080911B
:101EA0006A0086FF0AC0962FF901A2E7B0E084918C
:101EB0008D9331969150D9F708C0962FF901A2E77A
:101EC000B0E081918D939150E1F76150C901860F87
:101ED000911D6F5F019690938C0080938B00772704
:101EE000162F82E790E00EDD1C5F1C3010F01CE026
:101EF00003C08FEF809361001093600094E180B382
:101F00008C70B1F49150D9F710928E001092880025
:101F10000FC068506093610088E898279093710023
:101F200068E0B9CF60E082E790E0ECDC14E0E1CF5C
:101F3000DF91CF911F910F91FF90EF90DF90CF90A5
:101F4000BF900895A99A959AE0E0F0E08491999B5A
:101F500002C0A998A19A8F5F823038F0DF0129D0A2
:101F6000802D823411F0859923C081E08BBF82E0FF
:101F70008BBF8CE081BB9EEF8FEF9150F1F78150CA
:101F8000E1F711BA85B7826085BF8BB780648BBFDC
:101F90008BE480937D008AE580937C0078941DDE3D
:101FA000809170008823D9F31FEF17DE1150E9F7F5
:101FB0000ADEE199FECFBFBBAEBBE09A11960DB22F
:041FC0000895FFCFB2
:0A1FC4005AFFFF014000002000005A
:0400000300001800E1
:00000001FF
